:020000020000FC
:020000000BC033
:02000600CBC26B
:10001600A5C24FE54DBF44E04EBF4FEF47BB44BBC3
:1000260042BB4AE743BD41EC4FBD41E04EBD40E80F
:100036004ABD4AE045BD40E849BF60B3669566954E
:10004600669566956695603011F4B3E0A0E461307C
:1000560011F4B1E0A0EA623011F4B0E0AFEC633025
:1000660011F4B0E0A7E6643011F4B0E0A3E3653024
:1000760011F4B0E0A2E2663011F4B0E0ACE1673012
:1000860011F4B0E0A0E1B0BDA9B940E94AB9DD2458
:10009600CC247727C0EAD3E040E0499353E0C43B41
:1000A600D507D9F7C0E6D0E040E2499353E0C0381F
:1000B600D507D9F7C5E0D1E049EC49934DEC499312
:1000C600499349934993499349934993499349934A
:1000D600499349934993499349934993499349933A
:1000E600499349934993499349934993499349932A
:1000F6004993499349934BEB4993CDE2D1E04AEBBF
:100106004993CAE4D1E04993C5E5D1E04993C2E7F2
:10011600D1E04993CDE7D1E04993CAE9D1E04993CB
:10012600C5EAD1E04993C2ECD1E04993CDECD1E0E8
:100136004993CAEED1E04993C5EFD1E04993C2E1B4
:10014600D2E04993CDE1D2E04993CAE3D2E04993A4
:10015600C5E4D2E04993C2E6D2E04993CDE6D2E0C7
:1001660048EC49934DEC49934993499349934993F4
:100176004993499349934993499349934993499399
:100186004993499349934993499349934993499389
:1001960049934993499349934993499349934CEB1E
:1001A6004993C9E5D1E043E3499342E3499340E3E8
:1001B600499348E7499342E3499344E3499340E32B
:1001C600499340E249934CE4499343E4499344E418
:1001D600499340E2499343E449934FE649934EE6F7
:1001E600499344E7499342E749934FE649934CE6DE
:1001F60049934CE6499345E6499342E74993CEEA4B
:10020600D1E044E3499340E3499348E7499342E305
:10021600499340E3499340E249934AE5499345E6C9
:10022600499349E6499343E6499348E6499345E6A7
:1002360049934EE64993CEEFD1E048EB499340E22D
:10024600499342E6499349E7499340E2499342E498
:10025600499345E649934EE6499345E6499344E674
:10026600499349E649934BE6499344E74993C0E5E8
:10027600D2E0603051F440E3499341E3499342E3CD
:10028600499340E3499340E34993613051F440E395
:10029600499342E3499344E3499340E3499340E356
:1002A6004993623051F440E3499344E3499348E368
:1002B600499340E3499340E34993633051F440E363
:1002C600499349E3499346E3499340E3499340E31D
:1002D6004993643051F441E3499349E3499342E336
:1002E600499340E3499340E34993653051F442E32F
:1002F600499348E3499348E3499340E3499340E3EC
:100306004993663051F443E3499344E3499348E300
:10031600499340E3499340E34993673051F445E3F9
:10032600499347E3499346E3499340E3499340E3BE
:10033600499340E2499342E4499341E6499345E7AC
:10034600499344E64993A0E6B0E07894C59ACD1463
:10035600F1F340E2C0E6D0E0499353E0C038D50758
:10036600D9F7C0E6D0E002D07460FDCFE8D07B7F3D
:10037600603278F070FD6882699343E0C038D40734
:1003860010F0C0E6D0E070FF089568804BED48831A
:100396000895613051F470FD6882C0E6D0E070FFC8
:1003A600089568804BED48830895623011F4C5982E
:1003B6000895633011F4C59A0895643021F470FDF0
:1003C60068827E7E0895663039F470FF68807160B9
:1003D6007F7E4BED48830895673031F470FF688067
:1003E60071614BED4883089570FD6882683091F421
:1003F60070FD6882C150D04040E0C036D40710F48A
:10040600C0E6D0E040E2488370FF089568804BED77
:10041600488308956A3081F470FD6882C85DDF4FB5
:1004260043E0C038D40710F0C0E6D0E070FF08956E
:1004360068804BED488308956B3049F440E2488369
:1004460070FF089540E2642E4BED488308956C30AA
:1004560089F4C0E6D0E040E253E04993C038D507BE
:10046600E1F7C0E6D0E070FF089540E2642E4BED60
:10047600488308956D3091F470FD688248E553E035
:10048600C417D50718F448525040FACFC42FD52FB9
:1004960070FF089568804BED488308956E3011F41F
:1004A6004ED008956F3049F44AD0653608F064E6B8
:1004B600462F660F4695640F6ABD6131D1F470FD13
:1004C60068823DD0462F3BD058E2659FD12DC02D86
:1004D600C05ADF4FC40F40E0D41F43E0C038D407F2
:1004E60010F0C0E6D0E070FF089568804BED4883B9
:1004F60008956E3189F470FD688221D020D0699309
:1005060043E0C038D40710F0C0E6D0E070FF08958D
:1005160068804BED488308956F3181F4CF93DF9364
:10052600C0EAD3E00CD0643108F060E0C60F66275D
:10053600D61F05D06883DF91CF9108950895CD1415
:10054600F1F35E01D3946D2D6F71D62E6627C0E848
:10055600D3E0CD0DD61F6881E50108952FB60CB105
:10056600C3941C2D1F711D1539F0C12E1127A0E84B
:10057600B3E0AC0DB11F0C932FBE189538BAED91B0
:10058600049148BA009505BB38BA029505BB48BA2E
:100596005A94A1F738BA17C02FB608E2502E08B3FE
:1005A6000E7F302E0160402ED701882039F738BAE9
:1005B600ED91049148BA05BB38BA029505BB48BA15
:1005C6005A94A9F738BAC29A3A9500000000C29820
:1005D60000000000C39819F0F39598971AC03CE004
:1005E6002395E0EAF3E00027E20FF01F8080F8E0B1
:1005F600243179F4C49BC49AB499C498C39A222727
:10060600A0E6B0E08090A0037A9419F402E2702E7E
:10061600726074FF0CC071FF0AC072FF08C07D7F54
:1006260073FF68820BED73FD088308E070277D0178
:040636002FBE189526
:1008000000000000000000000000000000000000E8
:1008100000000000000000000000000000000000D8
:1008200000000000030000000000000000000000C5
:1008300000000000000000000000000000000000B8
:1008400000000000000000000000000000000000A8
:100850000000000000000000000000000000010097
:100860000300000000000000000000000000000085
:100870000000000000000000000000000000000078
:100880000000C003000C830003000C000106008779
:10089000C0000003000C030C0000CC00C30000E00B
:1008A000C0C0C0C0006700000000000000000000E1
:1008B0004255D68181C08706006666006600CC007E
:1008C0008181008100810067660066006600660025
:1008D000CC00870006008187008100FF000006FF32
:1008E000810087060067000000818706608100C0E4
:1008F0000000000E000000000000000000000000EA
:1009000000E7E70001818100000000E3C300F70079
:1009100008208166F7E70081818100000000000067
:10092000000366C603000703C006000000000000C5
:10093000C7018787C0CF83EF87870000C000068785
:10094000C703CFC38FEFEFC3CC87E16E0F6C6C830F
:10095000CF83CF87CFCCCC6CCCCCEFC300C383008C
:1009600003000E00C10083000E81C00E870000004E
:100970000000000000000000000000C1810E3700F0
:1009800087CC8187CC06C60087CC06C68303CCCC37
:100990008100E387CC06870666CC000066A300B121
:1009A0008181818167CD878703830026360300001C
:1009B00029AABD818181CC03836666006603CC00D1
:1009C00081810081008167CD660066006600660057
:1009D000038FCCCC030F03CCCC8100FF008103FF3D
:1009E0000387CC0367CD00000F03CC03C003CF8186
:1009F00000000033F7E70000C3CC00038787000046
:100A0000003CFF4483C3C300000000E06600368161
:100A10000C60C366BD3600C3C3810000000001EF57
:100A2000008766C6C7008D03810300000000002018
:100A30006C03CCCCC10C066CCCCC0000810003CC88
:100A40006C876666C6266666CC03C06606EE6CC614
:100A500066C666CC4BCCCC6CCCCCEC0308C0C600D4
:100A600081000600C000C6000681C00681000000AB
:100A70000000000002000000000000038103AD0040
:100A8000CCCC03CCCC03C600CCCC03C6C68100CCF6
:100A9000000087CCCC03CC036600CC0006C60081E6
:100AA00003030303CD00CCCC0344006E6E030000AF
:100AB00094556B8181000000446666006603CC009B
:100AC000818100810081CD006600660066006600BD
:100AD0008DC6000000030000008100FF008100FFC0
:100AE00000CC0000CD00000E0600000081000003D5
:100AF00000030066BD36030066000007C0C00000AA
:100B00000018FFEEC7C3E700000000A36600F7BDB2
:100B10000EE0E766BD0300E7E7818103004201EFD5
:100B2000008766EF0C4C8D03038166810000006036
:100B3000EC0FCCC0C30C0C6CCCCC8383030081C005
:100B40006CCC666C6606266CCC03C0C606EF6E6C79
:100B5000666C66CC03CCCC6CCCCC89030CC06C002E
:100B600000000600C000060006000006810000002C
:100B70000000000006000000000000038103EC01FB
:100B8000CC0000000000830000000000000003878C
:100B9000CF008D00000000000087CC0006EC008133
:100BA00000000000006CCCCC00AB00C6C60000000A
:100BB00042AAD68181030303AB6666006687CC0038
:100BC0008181008100810003660066006600660086
:100BD000C066CFCFCF038787878100FF008187FF63
:100BE00087CC878700870006C7CCCCCC00CC000020
:100BF000000300C3BD030300660000038381CF0030
:100C0000005ABDEFEFFFFF0000000027660036E747
:100C10008FE38166BDC300818181C0060C6683C7F6
:100C2000008742C60CCC070606C0C381000000C086
:100C3000ED03C0C0C60C0C60CCCC838306E7C0813A
:100C4000EDCC660C6646460CCC03C0C606EF6F6C56
:100C5000666C660C03CCCC6C87CC810306C00000AC
:100C60000087C787C7870667C687C36681CF8F8718
:100C7000CD67CE87CFCCCC6C6C66CF0681810083EC
:100C80000CCC878787878F87878787878787878722
:100C90004CEF8D878787CCCC66CCCC87066D00E780
:100CA000878787CC8F6EE78703AA0087870333CCBB
:100CB0002955BD81818787872A6E66EF6ECC8700B4
:100CC000818100810081878776F77EFF76FF7E0035
:100CD00060664C4C4C030303038100FF008103FF5B
:100CE000CC8DCCCC87CC66C766CCCCCC66CC000097
:100CF00000CF008FBDC3000066000003C003CF001B
:100D00000018FFEFEF7EFF000000008FC300367E6B
:100D1000EFEF8166B76600818181EFEF0CFF83C73B
:100D2000000300C68781AF0006C0FFE700EF008127
:100D30006D038183CC8F8FC087C700000C006003D8
:100D4000EDCCC70C66C7C70CCF03C087066DEF6C30
:100D5000C76CC70703CCCC6D0387030303C0000037
:100D600000C066CCCCCC8FCC6781C0C6816DCCCCAA
:100D700066CCE6CC06CCCC6CC666C80C00C000C6FF
:100D80000CCCCCC0C0C0C0CCCCCCCC818181CCCC74
:100D90000CB1EFCCCCCCCCCC66CCCCCCCF6D6C81B8
:100DA000C081CCCCCC6F000006ABCF03730366666A
:100DB00094AA6B818FCCCCCC2A606660600CCF8FFC
:100DC000F1FFFFF1FFFFC0CC060600000600006C3B
:100DD000E76F0C0C0CCF0303038FF1FF000003FF40
:100DE000CCCCCCCCCCCC666666CCCCCC66CC000073
:100DF000CF038F73B766CF00C300818787C7CF004B
:100E000000DB3CEFC77EE700000000CC8100367EAF
:100E10008FE38100B16600818181C0060C66C783C3
:100E2000000300C6C003ED0006C0C381000000033C
:100E30006F0303C0EFC0CC81CC81000006E7C00384
:100E4000EDCF660C664646ECCC03CCC6266CED6C4A
:100E500006ECC68103CCCC6D8703060381C000007D
:100E600000C7660CCCCF06CC6681C087816DCCCC28
:100E700066CC670606CCCC6D836681068181006CEA
:100E80000CCCCFC7C7C7C70CCFCFCF818181CCCC0B
:100E90008FF78DCCCCCCCCCC66CCCCCD066DC681BE
:100EA000C781CCCCCCEDEFEF0C2BC0E6F687CC3372
:100EB0004255D68181CCCCCC2A606660600C03811F
:100EC000000081810081C7CC06060000060000C733
:100ED0006C668F8F8F000303030081FFFF81030087
:100EE000CCCCCCCCCCCC666666CCCCCC66870000B7
:100EF000000300F6B1660000000000000000CF0013
:100F000000997EC783818100000000CCE70076E76E
:100F10000EE0E700B1C3EFE781E78103EF42C7834B
:100F2000000000EFC006CC000381668100000006CF
:100F30006E0306C0C0C0CC03CC8183830300810054
:100F40000CCC666C6606066CCC03CCC6666CEC6C8E
:100F500006ED66CC03CCCCC6CC032603C0C0000093
:100F600000CC660CCC0C06CC6681C0C6816DCCCCA6
:100F700066CC068106CCCC6D836606038103006CCB
:100F8000CCCC0CCCCCCCCC0C0C0C0C818181CFCF3C
:100F90000C8D8DCCCCCCCCCC66CCCCCE066E8381EB
:100FA000CC81CCCCCCEC00000CAAC03CBD87CC33AF
:100FB00029AABD8181CFCFCFAB6E666EEFCCCF813A
:100FC000000081810081CCCFF776FF7E76FF7EC660
:100FD0006C660C0C0C000303030081FFFF8103000F
:100FE000CCCCCCCCCCCC66C7C7CCCCCC6603000078
:100FF000000000BDB1C30300000000000000CF00EE
:10100000003CFF8301818100000000CC81007EBD97
:101010000C60C366B1C0EFC381C300000000EF01E4
:10102000000300C68FCCCD00810300008300830C39
:101030006C03CCCCC0CCCC03CC03838381000303F2
:101040000CCC6666C6260666CC03CC66666C6CC69F
:1010500006C766CC03CC87C6CC036C0360C0000017
:1010600000CC66CCCCCC06C76681C066816DCCCC8A
:1010700066CC06CCC6CC87C6C6C34C03810300EF42
:10108000CCCCCCCCCCCCCCCC0C0C0C818181CCCCC1
:101090004C8D8DCCCCCCCCCCC3CCCCCC0CC6C68DA2
:1010A000CC81CCCCCC6C0000CC44C0683B8766665D
:1010B00094556B8181CCCCCC4466666600870381F5
:1010C000000081810081CCCC00660066660066C7A6
:1010D0006CC64C4C4C000303030081FFFF810300EE
:1010E000CC8FCCCCCCCC660606CCCCCCC3030000D9
:1010F00000CF8F3BB1C00300000000000000CF0014
:1011000000E7E70100E7E7000000008781006E814B
:1011100008208166B16CEF81818100000000EF0141
:10112000000300C603C86700C006000083008308F0
:10113000C7CFCF87E187870387070081C0000603F9
:10114000C7CCCFC38FEF0FE3CC87876EEF6C6C8378
:101150000FC06E87878703C6CC87EFC320C300000C
:101160000067CD8767870FC06EE7CC6EE76CCC87D2
:10117000C7C70F87836703C66CC0CFC1810E00004D
:101180008767876767676787C7C7C7E7E7E7CCCC25
:10119000CFFEED8787876767C0878787EF8B6C07F0
:1011A00067E78767CC6C0000878300C0F30333CC0C
:1011B00042AAD68181CCCCCC8366666600030381CB
:1011C00000008181008167CC006600666600666C65
:1011D000C78FCFCFCF008787870081FFFF81870030
:1011E000870C87878787B70F0F878787C08700009F
:1011F000000000F3B16C00000000000000000000DF
:1012000000000000000000000000000000000C00D2
:101210000000000000E700E7000000000000000000
:1012200000000000030000000000000006000000B5
:1012300000000000000000000000000300000000AB
:10124000000000000000000000000000000000009E
:1012500000E100000000000000000000000000FFAE
:1012600000000000000000CC0000CC0000000000E6
:1012700006C0000000000000008100000000000027
:101280000300000000000003000000000000000058
:1012900000000000000000008100000000000000CD
:1012A0000000000000000000000000F1300000001D
:1012B0002955BD818100000000666666000300813B
:1012C0000000818100810000006600666600660003
:1012D0000000000000000000000081FFFF0000008F
:1012E0000006000000000600000000008100000071
:1012F0000000003000E700030000000000000000D4
:1013000000000000000000000000000000000000DD
:1013100000000000000000000000000000000000CD
:1013200000000000000000000000000000000000BD
:1013300000000000000000000000000000000000AD
:10134000000000000000000000000000000000009D
:10135000000000000000000000000000000000008D
:10136000000000000000008700008700000000006F
:101370000FE1000000000000000F0000000000006E
:101380000600000000000006000000000000000051
:1013900000000000000000000F000000000000003E
:1013A000000000000000000000000000000000003D
:1013B00094AA6B81810000000066666600000081CF
:1013C0000000818100810000006600666600660002
:1013D0000000000000000000000081FFFF0000008E
:1013E0000000000000000C00000000000F000000E2
:1013F00000000000000000070000000000000000E6
:00000001FF
